:1000000000308A001E2B00000A108A100A11820795
:1000100028340C34013406340A108A100A1182077D
:100020002034203445343D34253434342E343234B5
:10003000663420346C34783420340A3400340A10A6
:100040008A100A1182072034203472346F347A34D3
:10005000733461346834203431340A340D3400345C
:100060000A108A100A1182072034203445343D34A6
:10007000253433342E343134663420346C347834BF
:1000800020340A3400340A108A100A1182072034FE
:10009000203472346F347A347334613468342034E9
:1000A00032340A340D3400340A108A100A118207DF
:1000B0002034203445343D34253434342E34303427
:1000C000663420346C34783420340A3400340A1016
:1000D0008A100A1182072034203472346F347A3443
:1000E000733461346834203433340A340D340034CA
:1000F0000A108A100A1182072034203445343D3416
:10010000253433342E343134663420346B346C343B
:10011000783420340A3400340A108A100A11820715
:100120002034203472346F347A3473346134683458
:10013000203434340A340D3400343A3084008313CC
:1001400000080319B4280130F800BF30F70064003C
:10015000F70BA728F80BA5284A30F700F70BAE28B5
:1001600000006400800BA328003407080F39C20088
:10017000400EF700F030F7057708F03942048700A9
:1001800006148316061064008312061083160610E8
:1001900083120034BE08031DCF288610D028861491
:1001A000831686108312BF0E3F08C000B520BF0E15
:1001B0003F08C000B52064000C30F700F70BDE28C4
:1001C000E12800341430BA009D200F3083168705D3
:1001D000831286108316861083120610831606106B
:1001E0008312A7012708023C031CFE280230BA0034
:1001F0009D200330C000B520A70AF22864000C300F
:10020000F700F70B012904290230C000B520640073
:100210000C30F700F70B0A290D29A7012708023C2B
:10022000031C1E2927080420A800BE012808BF00BF
:10023000CA200230BA009D20A70A0E29792B8E30E1
:10024000F7002808F8002708F900FA01F808031D4C
:1002500033297908F800F9010830F702F808031D7E
:100260003329F7013B290310F81B3A29F90DF80D42
:10027000F7033329F8138D2B39080319AC29C10072
:100280003D080319AC29C10703184D297F30C1026D
:10029000031CAC290319AC2951298130C10703186B
:1002A000AC294108F700F801F901FA013A08C50044
:1002B000C5173B08C4003C08C3001830C100C20188
:1002C000431C7A294008FA07031C6C29F90A031D0C
:1002D0006C29F80A0319C2173F08F907031C732990
:1002E000F80A0319C2173E08BB00BB173B08F80702
:1002F0000318C217C20DF80CF90CFA0CC50CC40C8B
:10030000C30C0310C10B5F290130F7070318AC2998
:10031000F81B9129C50DFA0DF90DF80DF703031916
:10032000AC29C51FA229FA0A031DA229F90A031D37
:10033000A229F80A031DA229F80CF90CFA0CF70AF5
:100340000319AC293A08C2003E08C206C21FAA29F6
:10035000F817B029F813B029F701F801F901FA01EB
:10036000003401303A02BC003B08023C031DBA29AC
:100370004030BC073C088038BD00BE013D08BF00CE
:10038000CA20003439080C3A0319D029063A031957
:10039000D829073A0319DE29053A0319E329E82980
:1003A000BE010130BF00CA200230BA009D20F429EE
:1003B0000130BA000230BB00B121F4290130BA008B
:1003C000BB00B121F429BE011030BF00CA20F429BE
:1003D00039081F3C031CEE290730B9050130BE0067
:1003E0003908BF00CA20F4290034F701F801F901E7
:1003F000FA01C101C201C301C40140083F043E0427
:100400003D040319332A2030C5000310B90DBA0D7D
:10041000BB0DBC0DC10DC20DC30DC40D400844027F
:10042000031D1C2A3F084302031D1C2A3E084202EA
:10043000031D1C2A3D084102031C2D2A3D08C10250
:100440003E08031C3E0FC2023F08031C3F0FC302BD
:100450004008031C400FC4020314F70DF80DF90DFA
:10046000FA0DC50B052A41308400831300340408BB
:10047000B1003008B3000319562A2F08BC002E081B
:10048000BB002D08BA002C08B900C001BF01203004
:10049000BE008230BD003C217A08AF007908AE0072
:1004A0007808AD007708AC00B30B3D2A2F08BC00DC
:1004B0002E08BB002D08BA002C08B9003908B63C3C
:1004C000B900FA013A08BD00BA170310BA0CBB0C08
:1004D000BC0CFA0CF90CF80CF70CB90B652ABD1F13
:1004E0007C2AF709F809F909FA09F70A0319F80A41
:1004F0000319F90A0319FA0A7A08AF007908AE005D
:100500007808AD007708AC00AF1F932AB103B1168D
:10051000AC09AD09AE09AF09AC0A0319AD0A03195C
:10052000AE0A0319AF0A3B30B8009A30B700CA30A0
:10053000B600B5010A30B30030080319B10A2F081C
:10054000BC002E08BB002D08BA002C08B9003808E2
:10055000C0003708BF003608BE003508BD00F521D1
:100560000008AC00840A0008AD00840A0008AE0050
:10057000840A0008AF00FD308407F708031DD32A62
:10058000300A33020319D32A31080319D52A0F3947
:1005900033020319CD2A0318052BB11B052B311B80
:1005A000D52A2030012B2030B105B11EE32AB1122B
:1005B0003008031DB1037708B1002D30B900C22106
:1005C0003108F700B10130083302031DF12A770822
:1005D000B1002E30B900C2213108F7002030B1053A
:1005E00000303030B11E012BB1123008031DB103B1
:1005F0007708B1002D30B900C2213108F700B101F0
:100600003030F7077708B900C2213808BC00370836
:10061000BB003608BA003508B900C001BF01BE01F1
:100620000A30BD00F5217A08B8007908B7007808CB
:10063000B6007708B500B30B9F2A003484018313FA
:100640001F30830583161F149F141F159F11073039
:100650009C00FF308312A000831681131F149F1487
:100660001F159F151F1383121F139F1783169F17A4
:1006700083121F148316091283129412A0122008E9
:1006800083168700831220162008831687008312A2
:10069000A0112008831687000130831294000030D7
:1006A000831694000108C73908388100831290012D
:1006B0000030F800920000308316920007309C0052
:1006C000050864000230F700F70B642B672B1C0849
:1006D00083120D1383169D010030F80083121F084A
:1006E000C73978049F0064000630F700F70B762BBB
:1006F000E2281F151F197A2B83161E088312A100EA
:100700001E08A2006400C730F700F70B852B00001D
:100710002208A8002108A7001F297A30BC00FF305A
:10072000BB001F30BA007930B9007A08C0007908E0
:10073000BF007808BE007708BD003C217A08A600FB
:100740007908A5007808A4007708A3008316061589
:1007500083120619E12BA70127080C20A70AF7002E
:10076000B900C22104302702031DAC2B03308400E2
:100770002608AF002508AE002408AD002308AC0011
:100780000230B00037220930A80028080C20A80A3F
:10079000F700B900C2210E302802031DC52BA701A6
:1007A00027081F20A70AF700B900C2210C30270232
:1007B000031DD02B0230A7009630BA009D20A70B56
:1007C000DC2B8316861583128619332CBC01BB01E2
:1007D0002030BA008230B9002608C0002508BF00CA
:1007E0002408BE002308BD003C217708A700780834
:1007F000A8007908A9007A08AA00AB012B083020CC
:10080000AB0AF700B900C22104302B02031DFE2BF6
:10081000023084002A08AF002908AE002808AD0085
:100820002708AC000130B00037220930AC002C089A
:100830003020AC0AF700B900C2210E302C02031D93
:10084000172CA70127084320A70AF700B900C221E7
:100850000C302702031D222C0230A7009630BA006C
:100860009D20A70B2E2C831606168312061A842CA5
:10087000BC01BB014830BA008530B9002608C00071
:100880002508BF002408BE002308BD003C217708CE
:10089000A7007808A8007908A9007A08AA00AB0187
:1008A0002B085420AB0AF700B900C22104302B02F8
:1008B000031D502C033084002A08AF002908AE0025
:1008C0002808AD002708AC00B00137220930AC0081
:1008D0002C085420AC0AF700B900C2210E302C02BB
:1008E000031D682CA70127086720A70AF700B90095
:1008F000C2210C302702031D732C0230A700963052
:10090000BA009D20A70B7F2C831686168312861AA9
:10091000BF2CA70127087820A70AF700B900C22139
:1009200004302702031D8A2C023084002608AF0001
:100930002508AE002408AD002308AC000130B0004B
:1009400037220930A80028087820A80AF700B90043
:10095000C2210F302802031DA32CA70127088C20D9
:10096000A70AF700B900C2210C302702031DAE2CE4
:100970000230A7009630BA009D20A70BBA2C831630
:0C09800006178312061FBF2C792B6300A2
:02400E00393F38
:00000001FF
